:020000000428D2
:08000800FF30A100FF30A2004F
:10001000FF30A300FF30A4000F30A5008A110A12A0
:1000200074230A308A110A12952326128A110A12A1
:10003000E12303308A110A12632332308A110A1233
:10004000B82303308A110A12632332308A110A124C
:10005000B82303308A110A12632332308A110A123C
:10006000B82332308A110A124D2328308A110A121D
:100070004D2323138A110A120324A3178A110A128B
:1000800000248A110A122224243098001930990081
:100090008A110A122524903098001A081A081A08A2
:1000A00000309900A3128A110A12062422138A1121
:1000B0000A120C24A2138A110A120924A7168A1103
:1000C0000A12DB2301308A110A128C23A7128A112B
:1000D0000A12DB23FF308A110A1215248A110A1230
:1000E0001F232808523C8A110A12031D7A288A11FC
:1000F0000A1282288A110A12F8225A08A8008A11C4
:100100000A1271288A110A12F8225A08A8008A11C4
:100110000A12F8225A08A8008A110A12F8225A086C
:10012000A8008A110A12F8225A08A8002808AA0072
:100130008A110A12F8225A08A8002808AB008A116E
:100140000A12F8225A08A8002808AC008A110A12DC
:10015000F8225A08A8002808AD008A110A12F822CD
:100160005A08A8002808AE008A110A12F8225A0874
:10017000A8002808AF008A110A12F8225A08A8001D
:100180008A110A12F8225A08A8008A110A12F822C3
:100190005A08A8008A110A12F8225A08A80028084A
:1001A000A9002908413C8A110A12031D2A2A8A1132
:1001B0000A12F8225A08A8008A110A12F8225A08CC
:1001C000A8002808B0008A110A12F8225A08A800CC
:1001D0002808B1008A110A12F8225A08A800280833
:1001E000B2008A110A12F8225A08A8002808B3009F
:1001F0008A110A12F8225A08A8002808B4008A11A5
:100200000A12F8225A08A8002808B5008A110A1212
:10021000F8225A08A8002808B6008A110A12F82203
:100220005A08A8002808B7008A110A12F8225A08AA
:10023000A8002808B8008A110A12F8225A08A80053
:100240008A110A12F8225A08A8002808B9008A114F
:100250000A12F8225A08A8008A110A12F8225A082B
:10026000A8002808BA008A110A12F8225A08A80021
:100270002808BB008A110A12F8225A08A800280888
:10028000BC008A110A12F8225A08A8002808BD00EA
:100290008A110A12F8225A08A8002808BE008A11FA
:1002A0000A12F8225A08A8002808BF008A110A1268
:1002B000F8225A08A8002808C0008A110A12F82259
:1002C0005A08A8002808C1008A110A12F8225A0800
:1002D000A8002808C2008A110A12F8225A08A800A9
:1002E0002808C3008A110A12F8225A08A8008A11A5
:1002F0000A12F8225A08A8002808C4008A110A1213
:10030000F8225A08A8008A110A12F8225A08A800EE
:100310002808C5008A110A12F8225A08A8002808DD
:10032000C6008A110A12F8225A08A8002808C70035
:100330008A110A12F8225A08A8002808C8008A114F
:100340000A12F8225A08A8002808C9008A110A12BD
:10035000F8225A08A8008A110A12F8225A08A8009E
:100360002808CA008A110A12F8225A08A800280888
:10037000CB008A110A12F8225A08A8002808CC00DB
:100380008A110A12F8225A08A8002808CD008A11FA
:100390000A12F8225A08A8002808CE008A110A1268
:1003A000F8225A08A8008A110A12F8225A08A8004E
:1003B0002808CF008A110A12F8225A08A800280833
:1003C000D0008A110A12F8225A08A8002808D10081
:1003D0008A110A12F8225A08A8002808D2008A11A5
:1003E0000A12F8225A08A8002808D3008A110A1213
:1003F000F8225A08A8002808D4008A110A12F82204
:100400005A08A8008A110A12F8225A08A8002808D7
:10041000D5008A110A12F8225A08A8002808D60026
:100420008A110A12F8225A08A8002808D7008A114F
:100430000A12F8225A08A8002808D8008A110A12BD
:10044000F8225A08A8008A110A12F8225A08A800AD
:100450002808D9002908413C8A110A12031DB22A32
:100460008A110A121B234C308A110A123F23613071
:100470008A110A123F2374308A110A123F233D3039
:100480008A110A123F2330088A110A123F233108C9
:100490008A110A123F23B0308A110A123F23320810
:1004A0008A110A123F2333088A110A123F233408A3
:1004B0008A110A123F2335088A110A123F2336088F
:1004C0008A110A123F2327308A110A123F23203053
:1004D0008A110A123F2339088A110A123F238A110E
:1004E0000A1217234C308A110A123F236F308A11E7
:1004F0000A123F236E308A110A123F233D308A11BF
:100500000A123F233A088A110A123F233B088A1134
:100510000A123F233C088A110A123F23B0308A1185
:100520000A123F233D088A110A123F233E088A110E
:100530000A123F233F088A110A123F2340088A11FA
:100540000A123F2341088A110A123F2327308A11D9
:100550000A123F2320308A110A123F2344088A11CD
:100560000A123F232908413C8A110A120319F22A70
:100570008A110A121F238A110A121B2320308A11A2
:100580000A123F2320308A110A123F2320308A1199
:100590000A123F2357308A110A123F2361308A1111
:1005A0000A123F2372308A110A123F236E308A11D9
:1005B0000A123F2369308A110A123F2367308A11D9
:1005C0000A123F2320308A110A123F2321308A1158
:1005D0000A123F2321308A110A123F2321308A1147
:1005E0000A123F238A110A1271288A110A12F52A67
:1005F000DA009818062B1819102B8C1EF92A8B1369
:100600008B1BFF2A1A088B17DA0008008B138B1B31
:10061000062B18121A081A081A0818168B17F92A26
:100620008B138B1B102B1A088B17F92A0800A83084
:100630008A110A124D2B80308A110A124D2B083074
:100640008A110A124D2301308A110A124D23C83033
:100650008A110A12B82302308A110A124D23C830B7
:100660008A110A12B82306308A110A124D230C305F
:100670008A110A124D23C8308A110A12B82BDA00E7
:1006800026168A110A12E1235A0E0F398A110A120C
:1006900063235A088A110A12632BDA0026128A1180
:1006A0000A12E1235A0E0F398A110A12632382308B
:1006B0008A110A12B8235A088A110A126323823057
:1006C0008A110A12B82BDB00A6168A110A12DE2341
:1006D0005B088A110A12E423A6128A110A12DE2389
:1006E000FA308A110A12CC2B00308A110A12E42344
:1006F00026128A110A12E123A6128A110A12DE2397
:1007000000308A110A12F52322128A110A121224C9
:10071000A2128A110A120F2CDA005A08DB00643088
:10072000DC000A308A110A129E2BA8002808DB0080
:100730006430DC0001308A110A129E2BDD00FF308C
:10074000DE005C08E0005B08DF0017308A110A1247
:100750005E070318A82B8A110A12DF0BA52B8A113A
:100760000A12E00BA32B8A110A12DD0BA12B080041
:10077000DB005B08DC00DC088A110A12031DC32BB6
:100780008A110A12CB2B0A308A110A12CC23DC03FD
:100790008A110A12BB2B0800DD00F430DE00FC30A9
:1007A000DF008A110A125D085E07031C00345F0730
:1007B0000318D72B08008A110A12EF2B8A110A128C
:1007C000F22B8A110A12F22BDC005C080F39DD00D3
:1007D0002608F0395D04A6008A110A12F22B2708B8
:1007E00087000800260886000800A80028080F399E
:1007F000A9002208F0392904A2008A110A121C2C2F
:100800008A110A12192C8A110A12192C8A110A1239
:10081000192C8A110A121C2C8A110A121C2C8A11FA
:100820000A121C2C8A110A121C2CA1008A110A120D
:100830001F2C230867000800220866000800210812
:1008400065000800831603130800831203130800D1
:02400E00723FFF
:00000001FF
